:100000000C94C5020C94E2020C94E2020C94E202FD
:100010000C94E2020C94E2020C94E2020C94E202D0
:100020000C94E2020C94E2020C94E2020C94E202C0
:100030000C94E2020C94E2020C947A070C94E20213
:100040000C94E2020C941A040C94BD030C947F03EC
:100050000C94E2020C94B90A0C94E2020C94E202B1
:100060000C94E2020C94E202756E6974203C2053F9
:1000700045525F434E5400626572746F732F637014
:10008000752F6176722F6472762F7365725F6D655E
:1000900067612E630073697A65203E2031006265D6
:1000A00072746F732F7374727563742F6669666FE1
:1000B0006275662E680066642D3E68772D3E727804
:1000C00062756666657200626572746F732F647222
:1000D000762F7365722E630066642D3E68772D3E21
:1000E000747862756666657200626572746F732FEC
:1000F0006472762F7365722E63002166642D3E69EB
:10010000735F6F70656E00626572746F732F6472D7
:10011000762F7365722E6300756E6974203C2063C0
:100120006F756E746F66287365725F68616E646C5C
:1001300065732900626572746F732F6472762F7312
:1001400065722E6300706F72742D3E69735F6F70FD
:10015000656E00626572746F732F6472762F7365BB
:10016000722E630066642D3E5F74797065203D3D9C
:10017000204B46545F53455249414C0062657274AE
:100180006F732F6472762F7365722E680021746905
:100190006D65725F696E697469616C697A65640026
:1001A000626572746F732F6472762F74696D6572F5
:1001B0002E63002674696D65722D3E6C696E6B004E
:1001C000626572746F732F6472762F74696D6572D5
:1001D0002E630066642D3E72656164006265727410
:1001E0006F732F696F2F6B66696C652E680066648C
:1001F0002D3E777269746500626572746F732F6942
:100200006F2F6B66696C652E68006368616E6E6542
:100210006C00626572746F732F6E65742F61783233
:10022000352E630063747800626572746F732F6E8D
:1002300065742F617832352E630066642D3E636CE1
:1002400065617265727200626572746F732F696F97
:100250002F6B66696C652E680066642D3E65727250
:100260006F7200626572746F732F696F2F6B6669AE
:100270006C652E68000000891112239B322446AD64
:10028000573665BF74488CC19D5AAFD3BE6CCAE562
:10029000DB7EE9F7F88110080193331A22A5562C6A
:1002A00047B7753E64C99C408DDBBF52AEEDDA6442
:1002B000CBFFF976E802218B30100299132667AF45
:1002C000763444BD554AADC3BC588ED19F6EEBE722
:1002D000FA7CC8F5D983310A2091121803A7772E2A
:1002E00066B5543C45CBBD42ACD99E508FEFFB6602
:1002F000EAFDD874C904428D5316619F702004A989
:10030000153227BB364CCEC5DF5EEDD7FC6888E1E1
:10031000997AABF3BA85520C4397711E60A11428E9
:1003200005B3373A26CDDE44CFDFFD56ECE99860C1
:1003300089FBBB72AA06638F7214409D512225ABC4
:10034000343006B9174EEFC7FE5CCCD5DD6AA9E3A1
:10035000B8788AF19B87730E6295501C41A3352AA9
:1003600024B1163807CFFF46EEDDDC54CDEBB96281
:10037000A8F99A708B088481951AA793B62CC2A508
:10038000D33EE1B7F04008C919522BDB3A644EED79
:100390005F766DFF7C899400859BB712A6ADD22451
:1003A000C3BFF136E0C1184809D33B5A2AE55E6C59
:1003B0004FF77D7E6C0AA583B4188691972EE3A72C
:1003C000F23CC0B5D14229CB38500AD91B666FEF39
:1003D0007E744CFD5D8BB502A499961087AFF32611
:1003E000E2BDD034C1C3394A28D11A580BE77F6E19
:1003F0006EF55C7C4D0CC685D71EE597F42880A170
:10040000913AA3B3B2444ACD5B5669DF78600CE9F8
:100410001D722FFB3E8DD604C79FF516E4A99020D0
:1004200081BBB332A2C55A4C4BD7795E68E11C68D8
:100430000DF33F7A2E0EE787F61CC495D52AA1A3AB
:10044000B03882B193466BCF7A5448DD59622DEBB8
:100450003C700EF91F8FF706E69DD414C5ABB12290
:10046000A0B9923083C77B4E6AD5585C49E33D6A98
:100470002CF11E780F6368203C3D2035004D6F64E1
:10048000656D2F68617264776172652E63006664C2
:100490002D3E5F74797065203D3D204B46545F4191
:1004A00046534B004D6F64656D2F6166736B2E680C
:1004B00000808183848687898A8C8E8F919294951F
:1004C00097989A9B9D9EA0A2A3A5A6A7A9AAACAD0A
:1004D000AFB0B2B3B5B6B7B9BABCBDBEC0C1C2C485
:1004E000C5C6C8C9CACBCDCECFD0D2D3D4D5D6D726
:1004F000D9DADBDCDDDEDFE0E1E2E3E4E5E6E7E8F4
:10050000E9EAEAEBECEDEEEEEFF0F1F1F2F3F3F401
:10051000F5F5F6F6F7F8F8F9F9FAFAFAFBFBFCFC50
:10052000FCFDFDFDFDFEFEFEFEFEFFFFFFFFFFFFEB
:10053000FF6275665F706F696E746572203E3D2064
:1005400062756600626572746F732F6D7761726594
:100550002F666F726D617477722E6300203D2030BC
:100560007825700A00496E76616C69642070747237
:100570003A20003A2000417373657274696F6E20EF
:100580006661696C65643A20000011241FBECFEFDC
:10059000D8E0DEBFCDBF11E0A0E0B1E0E0E9F8E3D4
:1005A00002C005900D92A836B107D9F716E0A8E66B
:1005B000B1E001C01D92A730B107E1F70E94410AE6
:1005C0000C94461C0C9400001092C00088E98093A3
:1005D000C10008951092C1000895FC0122852111E7
:1005E00005C021E0228788EB8093C10008959A011D
:1005F000AB01CA01B9019695879577956795605CBF
:100600007D4B804F9F4F0E94101C21503109309329
:10061000C5002093C4000895E2ECF0E08081A4E0DE
:10062000660F771FAA95E1F78F7C862B808308954C
:100630009FB7F89484B1886284B99FBF8FB7F8944C
:10064000229A8FBF8FB7F89424988FBF80ED8CBD0E
:100650008CB581608CBD8DB58E7F8DBD08951CBC21
:100660009FB7F89484B1837C84B99FBF089508959F
:100670000895FC01828508956FB7F894DC011A96FD
:100680002C911A97211120C0E0916205F091630529
:10069000478D50A121A132A142175307A9F021E0B3
:1006A0001A962C93A78DB0A185A196A1A817B9077A
:1006B00019F483A194A104C0A78DB0A1CD01019626
:1006C00090A3878F8C918EBD6FBF0895CF93DF93DA
:1006D000EC018230910544F049E953E067E770E0AE
:1006E00088E690E00E948C192BE02C9FC0012D9F82
:1006F000900D11248A5F9E4FDF91CF9108951F9234
:100700000F920FB60F9211242F933F938F939F93C5
:10071000AF93BF93EF93FF93E0916005F091610574
:10072000278D30A181A192A12817390731F488E9DA
:100730008093C1001092100113C0A78DB0A185A1B4
:1007400096A1A817B90719F483A194A104C0A78D95
:10075000B0A1CD01019690A3878F8C918093C600A4
:10076000FF91EF91BF91AF919F918F913F912F9109
:100770000F900FBE0F901F9018951F920F920FB6FB
:100780000F9211242F933F934F935F938F939F93D7
:10079000AF93BF93EF93FF93E0916005F0916105F4
:1007A00097A58091C0008871892B87A75091C600BA
:1007B00027A130A583A594A52817390739F421A5C9
:1007C00032A585A596A52817390761F021A532A580
:1007D00087A190A5019741E02817390709F040E06B
:1007E000842F01C081E080FF04C087A5816087A7B6
:1007F00012C0A1A5B2A55C9321A532A585A596A599
:100800002817390719F483A594A503C081A592A5DB
:10081000019692A781A7FF91EF91BF91AF919F9110
:100820008F915F914F913F912F910F900FBE0F903D
:100830001F9018951F920F920FB60F9211242F93AD
:100840003F934F938F939F93AF93BF93EF93FF93F8
:10085000E0916205F091630527A130A583A594A5D9
:100860002817390739F421A532A585A596A528179B
:10087000390761F021A532A587A190A5019741E034
:100880002817390709F040E0842F01C081E080FD7E
:1008900013C08EB5A1A5B2A58C9321A532A585A5BF
:1008A00096A52817390719F483A594A503C081A537
:1008B00092A5019692A781A7E0916205F091630548
:1008C000278D30A181A192A12817390799F0A78D12
:1008D000B0A185A196A1A817B90719F483A194A185
:1008E00004C0A78DB0A1CD01019690A3878F8C91F4
:1008F0008EBD02C010921B01FF91EF91BF91AF918D
:100900009F918F914F913F912F910F900FBE0F901C
:100910001F9018959FB7F89483E085BB14BC15BC55
:1009200082E084BD85B5836085BD16BC89EF87BD37
:10093000EEE6F0E080818E7F80838081826080831C
:100940009FBF0895CF93DF93EC01FB015FB7F8944D
:10095000278D30A183A194A128173907E9F421A19B
:1009600032A185A196A128173907B1F481E05FBFB4
:1009700080FD11C04FB7F894A1A1B2A1CC9321A1E1
:1009800032A185A196A12817390799F483A194A1D2
:1009900092A381A314C0DACF81A192A1278D30A1A7
:1009A0002150310941E08217930709F040E0842F7C
:1009B000DECF21A132A12F5F3F4F32A321A34FBF32
:1009C00080A991A9DC01ED91FC910084F185E02DD5
:1009D0000995CE019927DF91CF910895FC014FB77A
:1009E000F89427A130A581A592A54FBF28173907F4
:1009F00039F087A5897B79F024C087A5897BC9F761
:100A00004FB7F89427A130A581A592A54FBF28170D
:100A1000390799F3EECF2FB7F894A7A1B0A585A514
:100A200096A5A817B90719F483A594A504C0A7A192
:100A3000B0A5CD01019690A787A38C912FBF90E020
:100A400008958FEF9FEF0895AF92BF92CF92DF92FC
:100A5000EF92FF920F931F93CF93DF937C015B0183
:100A60006A01FC0100891189228933890C341245FD
:100A70002544334541F04CEB50E06CE771E084E6EF
:100A800091E00E948C19E50100E010E00C151D05B5
:100A900059F0C7010E94EE048F3F2FEF920721F01B
:100AA0000F5F1F4F8993F2CFC801DF91CF911F9144
:100AB0000F91FF90EF90DF90CF90BF90AF9008958F
:100AC000AF92BF92CF92DF92EF92FF920F931F935C
:100AD000CF93DF937C015B016A01FC0100891189DE
:100AE000228933890C3412452544334541F04CEBBF
:100AF00050E06CE771E084E691E00E948C19E5011A
:100B000000E010E00C151D0561F08991B7019927EF
:100B100087FD90950E94A204019619F00F5F1F4F68
:100B2000F1CFC801DF91CF911F910F91FF90EF900E
:100B3000DF90CF90BF90AF900895CF93DF93EC01FB
:100B4000488959896A897B894C3452456544734583
:100B500041F04CEB50E06CE771E084E691E00E94DC
:100B60008C198FA590E0DF91CF910895CF93DF93FB
:100B7000EC01488959896A897B894C34524565441E
:100B8000734541F04CEB50E06CE771E084E691E096
:100B90000E948C191FA6DF91CF910895CF93DF9308
:100BA000EC01488959896A897B894C3452456544EE
:100BB000734549F04CEB50E06CE771E084E691E05E
:100BC0000E948C1900C02F8D38A189A19AA12817E5
:100BD0003907C9F788A999A9DC01ED91FC91028434
:100BE000F385E02D09958111EECF80E090E0DF9153
:100BF000CF910895FC014FB7F89427A130A581A5A6
:100C000092A54FBF28173907B1F02FB7F894A7A1C5
:100C1000B0A585A596A5A817B90719F483A594A52D
:100C200004C0A7A1B0A5CD01019690A787A38C9180
:100C30002FBF90E008958FEF9FEF08956FB7F8945E
:100C4000FC0147A150A521A532A56FBF81E0421745
:100C5000530709F480E00895DC01D0968D919C91B2
:100C6000D197DC01ED91FC910480F581E02D099490
:100C7000EF92FF920F931F93CF93DF93EC018B01C1
:100C80006230710540F042E651E064E371E088E1D2
:100C900091E00E948C19F801EE0FFF1FE05AFA4F05
:100CA000D183C0838E8D882341F045E651E067E013
:100CB00071E08AEF90E00E948C1981E08E8F1D8F89
:100CC0000C8FC8010E94660399AB88ABDC011296B9
:100CD0008D919C911397892B41F44DE651E069EE7B
:100CE00070E088ED90E00E948C19E8A9F9A9848150
:100CF0009581892B41F44EE651E067EC70E086EB7C
:100D000090E00E948C19E8A9F9A9E680F780028199
:100D10001381B2E0EB16F10440F441E251E06EE9D8
:100D200070E085E990E00E948C191CA30BA31AA324
:100D300009A318A30F8FC7010197800F911F9EA3CE
:100D40008DA3E8A9F9A9E084F18404811581E2E08A
:100D5000EE16F10440F441E251E06EE970E085E9FD
:100D600090E00E948C191CA70BA71AA709A718A727
:100D70000FA3C7010197800F911F9EA78DA788A978
:100D800099A9DC01ED91FC910190F081E02DBE016B
:100D9000099540E855E260E070E0CE010E942C0623
:100DA0001FA6CE01DF91CF911F910F91FF90EF9081
:100DB00008954FB7F894FC0121A532A530A727A3C9
:100DC0004FBF08954FB7F894FC0121A132A130A381
:100DD000278F4FBF0895CF93DF93EC010E94D90670
:100DE000CE01DF91CF910C94E206CF93DF93EC011B
:100DF000488959896A897B894C34524565447345D1
:100E000041F04CEB50E06CE771E084E691E00E9429
:100E10008C198E8D811108C04BE851E063E571E0BB
:100E200085E491E00E948C191E8ECE010E94CE05B1
:100E300088A999A9DC01ED91FC910280F381E02D54
:100E4000099519AA18AACE010E94EB0680E090E04D
:100E5000DF91CF910895CF93DF93EC0148895989B1
:100E60006A897B894C3452456544734541F04CEBAB
:100E700050E06CE771E084E691E00E948C19CE01AD
:100E80000E94F5066C8D7D8DCE010E943806CE0144
:100E9000DF91CF910895FC01CB0122E3DF011D9288
:100EA0002A95E9F74CE452E565E473E5408B518BF4
:100EB000628B738B2BE237E03583248325EF36E09A
:100EC0003783268324E235E03183208320E635E032
:100ED000338322832EEC35E0338722872DE935E0FA
:100EE0003587248726EB35E037872687BC01CF017D
:100EF0000C9438061F920F920FB60F9211240F9385
:100F00001F932F933F934F935F936F937F938F9391
:100F10009F93AF93BF93CF93DF93EF93FF93809112
:100F2000640590916505A0916605B09167050196ED
:100F3000A11DB11D8093640590936505A09366057E
:100F4000B09367050BEA1AEBC091A801D091A901F3
:100F500088819981892BD1F18FB7F89440916405EC
:100F60005091650560916605709167058FBF888512
:100F70009985AA85BB85481B590B6A0B7B0B77FDAE
:100F800025C0CF3FD10509F048F42BEC30E040EC10
:100F900051E063EB71E0CE010E94A219EA81FB816E
:100FA0008881998191838083E881F9818A819B81FD
:100FB000938382831B821A82198218821B8B0A8B6D
:100FC000EC85FD85CE010C960995BECFFF91EF9182
:100FD000DF91CF91BF91AF919F918F917F916F9151
:100FE0005F914F913F912F911F910F910F900FBEE5
:100FF0000F901F9018958CEA91E09093A90180932F
:10100000A8011092AB011092AA011092AD011092AA
:10101000AC0188EA91E09093AF018093AE01109209
:1010200064051092650510926605109267050E948E
:101030008A0480916805882341F041E951E060EA23
:1010400071E08DE891E00E948C1981E08093680541
:101050000895EF92FF920F931F93CF93DF931F9208
:10106000CDB7DEB77C018B018983DB0112968D91B0
:101070009C911397892B41F44EE051E068EF71E0A9
:101080008EEE91E00E948C19D8011296ED91FC91A0
:10109000139741E050E0BE016F5F7F4FC801099593
:1010A000019719F4C701992702C08FEF9FEF0F90A6
:1010B000DF91CF911F910F91FF90EF9008950F93C3
:1010C0001F93CF93DF931F92CDB7DEB78C01DC0166
:1010D0008D919C91892B41F442EF50E06CED71E0D1
:1010E00083ED91E00E948C19D801ED91FC9141E0D3
:1010F00050E0BE016F5F7F4FC8010995019719F459
:10110000898190E002C08FEF9FEF0F90DF91CF9128
:101110001F910F910895CF92DF92EF92FF920F935C
:101120001F93CF93DF931F92CDB7DEB77C01462F7D
:1011300082E8860F9701265B3E4F6901823010F0EE
:101140006B3149F4F601608171818BE190E0498354
:101150000E9429084981D701A05BBE4F2C911196AE
:101160005C911197842F90E0FC01E227EE0FFF1FA6
:10117000EB58FD4F25913491052F10E020273127A2
:101180002D933C93F601608171810F90DF91CF9197
:101190001F910F91FF90EF90DF90CF900C94290852
:1011A0003F924F925F926F927F928F929F92AF92F7
:1011B000BF92CF92DF92EF92FF920F931F93CF9344
:1011C000DF933C016C0126EBC21A2EEFD20A5C01C0
:1011D0004BEAA41A4EEFB40AEC01CC5ADE4F8C0154
:1011E000045B1E4F7C0182EBE81A8EEFF80A332471
:1011F000339444244A94542C4301AEEA8A1AAEEF45
:101200009A0AF601808191810E945F088F3FFFEF6B
:101210009F0709F458C0D5012C91211128C08E37A1
:101220009105D1F4F80180819181429768F0D7014E
:101230008D919C91883B904F39F4D401ED91FC91B4
:10124000309711F0C30109953882F701518240822D
:10125000D8011D921C92D5CF8F37910511F41882B9
:10126000D0CF8B31910519F4F5013082CACF288196
:10127000222331F1D8012D913C912A34B1E03B0772
:10128000F0F4A9014F5F5F4FF80151834083F301F0
:10129000E20FF31F8083D7012D913C911197F90143
:1012A000E827FF27EE0FFF1FEB58FD4F8591949124
:1012B000232F3327822793278D939C9301C0188275
:1012C000F50110829ECFD601CD91DC918C859D8554
:1012D000892B41F449E451E063E672E089E592E04C
:1012E0000E948C19EC85FD85CE010995892B21F191
:1012F000F601C081D1818E859F85892B41F442E51D
:1013000051E067E472E08AE392E00E948C19EE8576
:10131000FF85CE01DF91CF911F910F91FF90EF904C
:10132000DF90CF90BF90AF909F908F907F906F9005
:101330005F904F903F900994DF91CF911F910F9153
:10134000FF90EF90DF90CF90BF90AF909F908F90E5
:101350007F906F905F904F903F9008958F929F92F3
:10136000AF92BF92CF92DF92EF92FF920F931F93B3
:10137000CF93DF938C014B016A017C0180EBE81A6B
:101380008EEFF80A8FEF9FEFF7019183808358016A
:10139000F6EBAF1AFEEFBF0AF501608171818EE7AF
:1013A00090E00E942908E401C80CD91CCC15DD0589
:1013B00029F06991C8010E948B08F8CFF70160817C
:1013C000C1816095C8010E948B086C2F6095C8018F
:1013D0000E948B08F501608171818EE790E0DF91BA
:1013E000CF911F910F91FF90EF90DF90CF90BF9022
:1013F000AF909F908F900C942908EF92FF920F93DB
:101400001F93CF93DF93EC018B017A01009741F496
:1014100041E251E068E272E084E292E00E948C19BD
:101420000115110541F442E251E062E172E08AE007
:1014300092E00E948C1986E591E0FE019C011192D8
:1014400021503040E1F7FE01E65BFE4F118300833F
:10145000FE01EE5AFE4FF182E082FE01E05BFE4F9C
:101460008FEF9FEF91838083C25BDE4F99838883E8
:10147000DF91CF911F910F91FF90EF9008950C9401
:10148000251078940E94FB0760E070E081EB91E00A
:101490000E944B0740E855E260E070E081EB91E08C
:1014A0000E942C0686E08093C20060E070E089E331
:1014B00093E00E94950F4FE35AE069E373E083EEF7
:1014C00091E00E94FD0961EB71E083EE91E00E94E2
:1014D0001C1083EE91E00E94D00881EB91E00E9405
:1014E0001E068823B1F381EB91E00E94FA058093F8
:1014F000B0010E947A10EDCFCF93DF93EC0170938F
:101500001404609313048630910544F041E250E0E6
:101510006DE774E085E794E00E948C1910928000DA
:1015200089E18093810081E896E090938700809321
:1015300086008C2F806480937C0087B121E030E0AE
:1015400001C0220FCA95EAF7922F9095892387B997
:1015500088B1892388B980917E00822B80937E0098
:1015600087E080937B008CEE80937A00DF91CF91AF
:1015700008951F920F920FB60F9211242F933F934D
:101580004F935F936F937F938F939F93AF93BF938B
:10159000EF93FF9380E286BB6091780070917900B1
:1015A000769567957695679560588091130490912C
:1015B00014040E94AC0C80916A05882349F0809144
:1015C0001304909114040E947C0E807F886007C0F1
:1015D00080916905882311F088E801C080E88BB903
:1015E000FF91EF91BF91AF919F918F917F916F91FB
:1015F0005F914F913F912F910F900FBE0F901F90D1
:101600001895AF92BF92CF92DF92EF92FF920F9315
:101610001F93CF93DF936C01EB017A01DC015096AD
:101620000D911D912D913C9153970D341B442345F1
:10163000364441F04EE650E064EA74E08EE894E00F
:101640000E948C195E01CE018E0D9F1DF601EB5795
:10165000FF4FA816B90671F4C5018C1B9D0BDF91D5
:10166000CF911F910F91FF90EF90DF90CF90BF909F
:10167000AF9008956FB7F8944081518122813381F2
:101680006FBF4217530741F32FB7F894C09064051A
:10169000D0906505E0906605F09067052FBF6FB7A5
:1016A000F89440815181228133816FBF42175307E3
:1016B000A9F44FB7F8940091640510916505209145
:1016C0006605309167054FBF0C191D092E093F09AA
:1016D000101611061206130614F7BECF6FB7F89452
:1016E00020813181468157812417350719F44481BF
:1016F000558105C020813181A9014F5F5F4F518322
:101700004083D9012C916FBFD5012D935D01A1CFED
:101710002F923F924F925F926F927F928F929F9201
:10172000AF92BF92CF92DF92EF92FF920F931F93EF
:10173000CF93DF93EC017B016A0188899989AA899B
:10174000BB898D349B44A345B64441F04EE650E03E
:1017500064EA74E08EE894E00E948C1987013701F6
:101760006C0C7D1C222423946E0187E7C80ED11CCB
:1017700080E4482E512C90E4892E9FE1992EA12CD3
:10178000B12C0615170509F477C04FB7F8942FA5AB
:1017900038A98BA99CA92817390739F429A93AA98E
:1017A0008DA99EA92817390761F029A93AA98FA503
:1017B00098A9019751E02817390709F050E0852FC3
:1017C00001C081E04FBF80FDE0CFF80181918F0122
:1017D0004FB7F894E9A9FAA9808329A93AA98DA954
:1017E0009EA92817390719F48BA99CA903C089A9B8
:1017F0009AA901969AAB89AB4FBFF60180818111FE
:1018000021C05EA64DA61CA61BA61AA62082299A58
:10181000209120013091210140912201509123011A
:10182000A0EBB4E00E94F11B6056704F8F4F9F4FAA
:10183000A50194010E94101C3BA32AA35B9AF1E02E
:10184000F0936A053FB6F89420911C0130911D0178
:1018500040911E0150911F01A0EBB4E00E94F11BCA
:101860006056704F8F4F9F4FA50194010E94101C2E
:101870003DA32CA33FBE85CFC8018E199F09DF91E0
:10188000CF911F910F91FF90EF90DF90CF90BF907D
:10189000AF909F908F907F906F905F904F903F9010
:1018A0002F900895CF93DF93EC01488959896A8975
:1018B0007B894D345B446345764441F04EE650E00D
:1018C00064EA74E08EE894E00E948C19C958DF4FF6
:1018D00088818111FDCF80E090E0DF91CF91089564
:1018E000CF93DF93EC01488959896A897B894D340C
:1018F0005B446345764441F04EE650E064EA74E0B0
:101900008EE894E00E948C192FB7F894C852DF4FEC
:10191000888199812FBFDF91CF910895CF93DF9375
:10192000EC01488959896A897B894D345B44634558
:10193000764441F04EE650E064EA74E08EE894E0CC
:101940000E948C198FB7F894C852DF4F1982188201
:101950008FBFDF91CF910895EF92FF920F931F9366
:10196000CF93DF93FC018C0101531F4FD8014D91A0
:101970005C91DC01A353BF4F4D935C93DC01A858ED
:10198000BF4F8D919C91119716962D913C91179771
:101990008217930729F414962D913C91159706C050
:1019A0008D919C9111979C012F5F3F4F11963C9315
:1019B0002E93EC012881260290011124359527955C
:1019C00035952795E801398328837F01D3EDED0E06
:1019D000F11CE701888199818F010F521F4FE801A7
:1019E0009983888395958795840F951F820F931F00
:1019F000E70199838883AF014B525F4F21E01816AE
:101A000019060CF020E0EA018881880F822B888378
:101A100012968D919C911397EC01688312962D91EB
:101A20003C91139716968D919C911797281739071B
:101A300029F414968D919C91159705C012968D915D
:101A40009C911397019613969C938E931297DA01AB
:101A50009C91892F8695869589278370DF01AA52EC
:101A6000BF4F833039F48C91803214F48F5F01C002
:101A700081508C938C91885F8C9380340CF435C1A9
:101A80008F738C93DF01A952BF4F8C91880F977091
:101A90002BEF290F233010F0933009F481608C93E1
:101AA0009C91892F8695892780958170968D990FB5
:101AB000892B868F8E3709F04EC0DF01AB57BF4FA1
:101AC0002D913C91119714968D919C911597281703
:101AD000390759F412962D913C91139716968D91D2
:101AE0009C9117972817390779F012962D913C9100
:101AF00013978D919C911197019741E02817390711
:101B000009F040E0842F01C081E080FDDDC0129625
:101B1000CD91DC9113978EE7888312962D913C919D
:101B2000139716968D919C9117972817390729F4CA
:101B300014968D919C91159705C012968D919C914C
:101B40001397019613969C938E93129781E081A32D
:101B50002A9A41E0BCC0982F9F779F3719F411A2B1
:101B60002A98C3C091A1992309F4BFC0982F9F73ED
:101B70009E3309F4BAC080FF03C080A1806880A3AF
:101B8000878D8F5F878F90A1883008F4ACC0DF010C
:101B9000AB57BF4F82E8890F823018F09B3109F0B4
:101BA0004BC02D913C91119714968D919C91159756
:101BB0002817390759F412962D913C9113971696D0
:101BC0008D919C9117972817390779F012962D91CE
:101BD0003C9113978D919C911197019741E02817A3
:101BE000390709F040E0842F01C081E080FD20C06A
:101BF0001296CD91DC9113978BE1888312962D91EB
:101C00003C91139716968D919C9117972817390739
:101C100029F414968D919C91159705C012968D917B
:101C20009C911397019613969C938E93129704C0E0
:101C300011A22A9840E001C041E02D913C911197FA
:101C400014968D919C9115972817390759F412967F
:101C50002D913C91139716968D919C91179728176B
:101C6000390779F012962D913C9113978D919C91A3
:101C70001197019751E02817390709F050E0852F97
:101C800001C081E080FD20C080A11296CD91DC9141
:101C90001397888312962D913C91139716968D91E8
:101CA0009C9117972817390729F414968D919C91C8
:101CB000159705C012968D919C91139701961396D6
:101CC0009C938E93129703C011A22A9840E010A211
:101CD000178E41110AC0E852FF4F808191818160C7
:101CE0009183808302C0969590A3DF91CF911F913D
:101CF0000F91FF90EF900895DC0196968C91969746
:101D00008111EAC098968C9198978111A0C09F96F6
:101D10002D913C91D097D1968D919C91D297281777
:101D2000390739F494968D919C919597892B09F4F4
:101D30005CC099968C919997811103C09A961C92D8
:101D40009A9781E099968C93999792968D919C9110
:101D50009397009789F59F962D913C91D097D196B6
:101D60008D919C91D2972817390751F494968D91B3
:101D70009C919597019795969C938E93949721C0EB
:101D80009F96ED91FC91D097D5968D919C91D69789
:101D9000E817F90729F4D3968D919C91D49706C042
:101DA0009F96ED91FC91D097CF010196D0969C9390
:101DB0008E939F97808106C0019793969C938E93F4
:101DC00092978EE797968C93979797968C91979783
:101DD0008B3199F59F962D913C91D097D1968D910D
:101DE0009C91D2972817390749F45B9810926A059D
:101DF000A958BF4F1C92299880E008959F96ED91B5
:101E0000FC91D097D5968D919C91D697E817F907BC
:101E100029F4D3968D919C91D49706C09F96ED910D
:101E2000FC91D097CF010196D0969C938E939F976B
:101E3000808197968C93979706C08E57823018F4BE
:101E400099961C92999781E098968C939897999679
:101E50002C9199979D968D919C919E972223A9F004
:101E60009A962C919A97253080F09A961C929A9780
:101E70008034910519F485E790E002C080E490E099
:101E80009E969C938E939D9723C098963C9198978D
:101E900097962C919797232341F09A968C919A9735
:101EA0008F5F9A968C939A970FC09A961C929A97E6
:101EB0008034910519F485E790E002C080E490E059
:101EC0009E969C938E939D97330F98963C939897EC
:101ED00088E096968C9396979D96ED91FC919E97AF
:101EE0009B968D919C919C97E80FF91F9F013170F3
:101EF0009C963C932E939B9796968C9196978150A7
:101F000096968C93FF27E038F10530F08FEF90E044
:101F1000AC014E1B5F0BFA01EF54FB4F84912F3F36
:101F2000310511F008F080950895CF93DF93EC010F
:101F3000CB012AEDFE0111922A95E9F77D8F6C8F76
:101F400020E430E03EA72DA79E0120583F4FFE0120
:101F5000E858FF4F358324833383228331832083E2
:101F60009E012C573F4F378326839E0123573F4FB7
:101F7000DE01AB57BF4F15963C932E9314971396E3
:101F80003C932E93129711963C932E939E012453CB
:101F90003F4F17963C932E9316979E01295C3F4F17
:101FA0003CAB2BAB3AAB29AB38AB2FA79E012A58E1
:101FB0003F4F3EAB2DAB24E030E0A281B3811C92B9
:101FC00062817381468157816417750719F44481D2
:101FD000558104C0428153814F5F5F4F53834283D9
:101FE000215031092115310541F7BE010E947C0ABB
:101FF0008AB1886F8AB9219A229A4DE45BE463E53D
:1020000076E4488B598B6A8B7B8B88E89BE09B83BB
:102010008A8381E09BE09983888382E59CE09B87AB
:102020008A8780E79CE09D878C878EE89CE09F876D
:102030008E87DF91CF91089590939E0580939D05A3
:1020400070930206609301060895EF92FF920F933A
:102050001F93CF93DF93EC0160910106709102060C
:1020600080EC90E00E9429086091010670910206C0
:1020700080E090E00E9429088E017E0184EBE81A3E
:102080008EEFF80AF70180819181609101067091CD
:10209000020698012C1B3D0B2817390708F5F8019B
:1020A00081918F01803C59F48BED90E00E942908CA
:1020B00060910106709102068CED90E00EC08B3DA0
:1020C00059F48BED90E00E9429086091010670910F
:1020D00002068DED90E001C090E00E942908D2CF69
:1020E00080EC90E0DF91CF911F910F91FF90EF90E6
:1020F0000C942908282F809104068823A1F0203C05
:1021000001F580912401811111C0109204064091C3
:1021100005065091060665E174E080919D05909159
:102120009E050C94AE09203C09F061C081E08093CB
:1021300004068EEF80932401109206061092050685
:10214000089580910506909106068A3431E0930740
:1021500008F04DC030912401009731F43E3F21F446
:102160002F7020932401089531111FC02B3D21F4BD
:1021700081E080930306089530910306332349F0EC
:102180002C3D21F02D3D19F42BED01C020EC1092D7
:102190000306AC014F5F5F4F509306064093050660
:1021A000FC01EB5EFB4F20830895313071F430E089
:1021B000AAE0B0E00E94E21B60932001709321012D
:1021C00080932201909323010895343081F43AE002
:1021D000239FC0011124AA2797FDA095BA2F8093B1
:1021E0001C0190931D01A0931E01B0931F0108953F
:1021F0002F923F924F925F926F927F928F929F9217
:10220000AF92BF92CF92DF92EF92FF920F931F9304
:10221000CF93DF93CDB7DEB7C45AD1090FB6F89488
:10222000DEBF0FBECDBFC856DF4F99838883C85924
:10223000D040C656DF4F79836883CA59D040C45610
:10224000DF4F59834883CC59D0405901C257DF4FE3
:1022500019821882CE58D0409E012F5F3F4FC95738
:10226000DF4F39832883C758D040AE014A575F4FAC
:10227000C757DF4F59834883C958D040C856DF4FEE
:1022800008811981C859D0400F5F1F4FC856DF4FD2
:10229000E881F981C859D0408491853291F1882331
:1022A00009F448C7C456DF4F68817981CC59D040C2
:1022B000C656DF4FE881F981CA59D0400995C25707
:1022C000DF4FE880F980CE58D040FFEFEF1AFF0AC9
:1022D000C557DF4FB982A882CB58D040C856DF4FD0
:1022E00019830883C859D040C257DF4FF982E8826A
:1022F000CE58D040C557DF4FA880B980CB58D040CA
:10230000BDCFF8018491853259F5C856DF4F288139
:102310003981C859D0402E5F3F4FC856DF4F3983AF
:102320002883C859D040C456DF4F68817981CC5981
:10233000D040C656DF4FE881F981CA59D04009958F
:10234000C257DF4FE880F980CE58D040FFEFEF1A38
:10235000FF0AC557DF4FB982A882CB58D040C4CFFF
:10236000C256DF4F1882CE59D040C357DF4F188274
:10237000CD58D040C057DF4F1882C059D040CF56FB
:10238000DF4F1882C159D040F8012491C80101964D
:102390002B3209F458C060F42032E9F0233209F0FE
:1023A0005AC0F1E0C357DF4FF883CD58D04051C039
:1023B0002D3251F0203309F04EC021E0C256DF4FDC
:1023C0002883CE59D04045C0F1E0C057DF4FF88395
:1023D000C059D0403EC0232D2C7F322ECF56DF4F28
:1023E0003881C159D040332ACE56DF4F4881C25977
:1023F000D04040FB32F8C057DF4F5881C059D04021
:1024000050FB33F820FA34F8CD56DF4FA881C3597A
:10241000D040A0FB35F8C357DF4FB881CD58D0402E
:10242000B0FB36F8CC56DF4FE881C459D040E0FB12
:1024300037F8232D237069F441E0CF56DF4F4883EE
:10244000C159D04006C031E0CF56DF4F3883C15963
:10245000D0408C0199CFC357DF4F5881CD58D04021
:10246000C056DF4F5883C05AD040F80124912A3219
:1024700021F0612C712C3AE025C095012E5F3F4F71
:10248000D5016D907C9077FE09C0719461947108BC
:10249000B1E0C057DF4FB883C059D0408C0159011B
:1024A00016C02A33A0F40F5F1F4FFC018491A301D3
:1024B000349F3001359F700C112450E3651A710868
:1024C000680E711CC801F8012491203350F7C057E1
:1024D000DF4FF881C059D040FF2329F0C256DF4FAB
:1024E0001882CE59D040F80184918E3249F5319648
:1024F00084918A3229F08F01412C512C3AE01AC084
:10250000D5014D905C900E5F1F4FF50132965F0133
:102510001AC02A33C0F40F5F1F4FFC018491A2013F
:10252000349F2001359F500C112450E3451A510867
:10253000480E511CC801F8012491203350F703C004
:1025400044244A94542CF8012491C8010196283659
:1025500099F018F42C3439F017C02C3621F02A37B2
:1025600099F4212C02C0222423948C01CD56DF4FF4
:102570001882C359D0400EC08C01F1E0CD56DF4F18
:10258000F883C359D04005C0CD56DF4F1882C359D8
:10259000D040212C98012F5F3F4FC856DF4F398321
:1025A0002883C859D040F801D490C956DF4FD8824B
:1025B000C759D040F5E6DF1609F402C2FD15ECF06C
:1025C00023E5D21609F453C02D1564F035E4D31673
:1025D00009F4F6C147E4D41609F4E1C1DD2009F499
:1025E0006FC42AC053E6D51671F15D150CF4C6C050
:1025F00088E5D81609F48DC01FC090E7D91609F4F4
:1026000071C09D1564F0A7E6DA1609F4C8C1DA16A0
:102610000CF4D1C1B9E6DB1609F4B0C00DC0E5E792
:10262000DE1609F476C0F8E7DF1609F46DC023E77B
:10263000D21202C0F12C1DC0C557DF4FB982A8824B
:10264000CB58D04049C4A5014E5F5F4FC557DF4FFF
:1026500059834883CB58D040D5018C918983F12C84
:102660008E010E5F1F4FFE0131964F0143C4FF24C0
:10267000F39495012E5F3F4FC557DF4F3983288371
:10268000CB58D040D5018D909C908114910421F4B9
:10269000A9E28A2EA1E09A2E57FE04C0F0E14F2E47
:1026A000F7E25F2E8401FF20C1F0F80184918823B6
:1026B00009F420C4C80188199909841595050CF0FE
:1026C00019C40F5F1F4FF1CFC801881999098415EC
:1026D00095050CF00FC40F5F1F4FD8018C9181112D
:1026E000F3CF08C4F5013296C557DF4FF983E8836D
:1026F000CB58D040D5016D917C9180E090E0E8E42A
:10270000EE2EE1E0FE2E26C078E5E72E71E0F72EF2
:1027100004C068E4E62E61E0F62E222071F0F50197
:102720003496C557DF4FF983E883CB58D040D501A5
:102730006D917D918D919C910DC0C5010296F50121
:1027400060817181C557DF4F99838883CB58D04012
:1027500080E090E021E0CE56DF4F2883C259D04080
:1027600035E7D31205C0CE56DF4F1882C259D0408C
:10277000CF56DF4F1882C159D0403EC0222079F099
:10278000A5014C5F5F4FC557DF4F59834883CB5836
:10279000D040D5016D917D918D919C910FC0F50137
:1027A0003296C557DF4FF983E883CB58D040D50127
:1027B0006D917C91882777FD8095982F97FF13C0A6
:1027C00090958095709561957F4F8F4F9F4FCE5616
:1027D000DF4F1882C259D040B2E0CF56DF4FB883E6
:1027E000C159D04005C0CE56DF4F1882C259D040E3
:1027F00058E4E52E51E0F52EE1E0CC56DF4FE883BA
:10280000C459D040611571058105910529F4CC5654
:10281000DF4F1882C459D0404114510441F4CC56C2
:10282000DF4FF881C459D040FF2309F476C0CE565B
:10283000DF4F2881C259D0408E010A571F4F2130E7
:10284000A9F02AE030E040E050E00E94101CF701BF
:10285000E60FF71F8081D8018E938D01B901CA015F
:10286000611571058105910561F715C0FB01EF70D8
:10287000FF27EE0DFF1D2081F80122938F0144E018
:1028800096958795779567954A95D1F76115710566
:102890008105910559F757FE43C0C256DF4FF881B5
:1028A000CE59D040FF23E1F1232D2C7F322ECF567D
:1028B000DF4F3881C159D040332ACE56DF4F48818F
:1028C000C259D04040FB32F8C057DF4F5881C05941
:1028D000D04050FB33F820FA34F8CD56DF4F8881D2
:1028E000C359D04080FB35F8C357DF4F9881CD588E
:1028F000D04090FB36F8CC56DF4FA881C459D04069
:10290000A0FB37F8232D237081E090E011F480E0E4
:1029100090E02301481A590A03C08E010A571F4F3D
:10292000C757DF4F88819981C958D040801B910BD0
:10293000F80120E34F01841595051CF422930196BC
:10294000F9CFC357DF4FB881CD58D040BB23A1F09A
:10295000CC56DF4FE881C459D040EE2369F08D2D6D
:102960008F7D883549F4F4013197D082F2E08F1AD7
:10297000910880E3D4018C93C957DF4FE881F98136
:10298000C758D0408E169F0608F0AEC247EB52E003
:1029900064E475E081E395E00E948C19A5C2DA94A5
:1029A000DA94C956DF4FD882C759D04011E041149C
:1029B000510469F006C0C956DF4F1882C759D0408C
:1029C00010E057FE07C026E0422E512C03C04424DD
:1029D0004394512C95012C5F3F4FC557DF4F3983EE
:1029E0002883CB58D040D501CD90DD90ED90FC9060
:1029F00020E030E0A901C701B6010E942C1A87FF30
:102A00000AC0F7FAF094F7F8F094B2E0CF56DF4F2F
:102A1000B883C159D040C156DF4F1883CF59D04039
:102A200088248394912C8C0E9D1E860C971C20E08C
:102A300030E040E85FE3C701B6010E947B1B87FDE1
:102A400032C0A12CB12C27EB33E44AEB51E5C7018E
:102A5000B6010E947B1B87FD0EC029EF32E045E1E5
:102A600050E5C701B6010E94301A6B017C01EAE013
:102A7000AE0EB11CE8CF20E030E040E251E4C701E7
:102A8000B6010E947B1B87FD49C020E030E040E298
:102A900051E4C701B6010E94301A6B017C01FFEFBF
:102AA000AF1ABF0AE8CF20E030E0A901C701B601A4
:102AB0000E942C1AA12CB12C882381F12FEF36EE25
:102AC0004BED5EE2C701B6010E942C1A181674F095
:102AD00029EF32E045E150E5C701B6010E947F1BB6
:102AE0006B017C012AE0A21AB108E8CF20E030E0B7
:102AF00040E85FE3C701B6010E942C1A87FF0EC0B1
:102B000020E030E040E251E4C701B6010E947F1BA3
:102B10006B017C0131E0A31AB108E8CF112321F148
:102B2000A414B50464F44CEFA4164FEFB4063CF0C3
:102B30004A185B08C956DF4F1882C759D04051E088
:102B4000451A510881E0C357DF4F9881CD58D040D6
:102B50009827C156DF4F9883CF59D040A1E0C35783
:102B6000DF4FA883CD58D040C956DF4FB881C75931
:102B7000D040B1114CC0B7FE3EC080E3E1E0F0E0D0
:102B8000EC0FFD1FE60DF71D80834114510461F425
:102B9000C357DF4FE881CD58D040E11105C0F401A3
:102BA000319680E090E007C0F40132968EE2D401C5
:102BB00011968C93C20195012F5F3F4F280F391F4B
:102BC00040E38F018217930729F0009719F0419392
:102BD0000197F7CF920120953095A216B3060CF419
:102BE000D6C02C01E1E0F0E0CB56DF4FF983E8835B
:102BF000C559D0405CC0222733272A193B09CB5640
:102C0000DF4F39832883C559D040840150C08401E7
:102C1000CB56DF4F19821882C559D04048C0C70132
:102C2000B6010E94981ACF55DF4F688379838A8353
:102C30009B83C15AD040CF55DF4F48815981C15A3B
:102C4000D040BA01882777FD8095982F0E94CB1A33
:102C50009B01AC01C701B6010E94C71920E030E01A
:102C600040E251E40E947F1B6B017C0198012F5FC1
:102C70003F4FCF55DF4F8881C15AD040805DD8018A
:102C80008C93CB56DF4F88819981C559D0400196EE
:102C9000CB56DF4FE881F981C559D040EF2B91F039
:102CA000CB56DF4F99838883C559D0408901CB56D5
:102CB000DF4F28813981C559D040421653060CF0A8
:102CC000AECF14C04114510439F4C357DF4FF8811B
:102CD000CD58D040FF2339F098012E5F3F4FEEE2F0
:102CE000D8011196EC9381E090E0DACF20E030E05B
:102CF00040EA50E4C701B6010E947B1B87FD47C034
:102D0000F80181E090E030E322912E3251F0820F01
:102D10008A3321F0808380E090E003C0308381E03B
:102D200090E08E169F0680F3892B89F1C956DF4FFC
:102D30003881C759D0403323B9F0F8018E169F0669
:102D400078F4DF018E919D018E3239F4CF01029724
:102D5000DC018C918083F90101C080833197EECF33
:102D6000BFEFAB1ABB0A0BC00F5F1F4FF8018E16E7
:102D70009F0628F4DF018E918083FD01F8CF81E367
:102D8000E1E0F0E0EC0FFD1FE60DF71D8083C1567A
:102D9000DF4FE881CF59D040EE2349F0F80182910E
:102DA000803311F48F01FACF8E3209F48F01C956A6
:102DB000DF4FF881C759D040FF23B9F1D801FC9308
:102DC000C8010296B7FE07C02DE211962C93B1946C
:102DD000A194B10804C02BE2D80111962C938C0168
:102DE000065F1F4F20E030E02F5F3F4FF801319624
:102DF000C5016AE070E00E94FC1B805DD8018C93E5
:102E00005B016115710511F08F01EECF22303105A4
:102E1000DCF3E21BF30B199781918E93215031095A
:102E200012161306CCF309501109C256DF4FB881B0
:102E3000CE59D040BB2309F45CC0E32DEC7F3E2E7D
:102E4000CF56DF4FF881C159D0403F2ACE56DF4FD1
:102E50002881C259D04020FB32F8C057DF4F38815B
:102E6000C059D04030FB33F820FA34F8CD56DF4F4C
:102E70004881C359D04040FB35F8C056DF4F5881D8
:102E8000C05AD04050FB36F8CC56DF4F8881C45929
:102E9000D04080FB37F8232D237081E090E011F4BF
:102EA00080E090E09301281B390BF40140E34F01CF
:102EB000C8018E1B9F0B82179307DCF44293F7CF58
:102EC000C557DF4FB982A882CB58D040C856DF4FD4
:102ED00019830883C859D040F12C08E211E085E23B
:102EE000882E81E0982E06C0F12C8E010A571F4FC4
:102EF00001C0F12C0819190960167106DCF1932D37
:102F00009C7F392ECF56DF4FA881C159D0403A2A35
:102F1000CE56DF4FB881C259D040B0FB32F8C0570F
:102F2000DF4FE881C059D040E0FB33F820FA34F895
:102F3000CD56DF4FF881C359D040F0FB35F8C0566D
:102F4000DF4F2881C05AD04020FB36F8CC56DF4FE7
:102F50003881C459D04030FB37F86301C01AD10A18
:102F6000232D237081E090E011F480E090E0C81AF6
:102F7000D90A02C0C12CD12CC057DF4F4881C0599B
:102F8000D040411122C031E0C31AD108D7FC1DC086
:102F9000C456DF4F68817981CC59D04080E2C65653
:102FA000DF4FE881F981CA59D0400995C257DF4FF8
:102FB00028813981CE58D0402F5F3F4FC257DF4F15
:102FC00039832883CE58D040DECF432D4C7F342E1A
:102FD000CF56DF4F5881C159D040352ACE56DF4FEA
:102FE0008881C259D04080FB32F8C057DF4F9881AA
:102FF000C059D04090FB33F820FA34F8CD56DF4F5B
:10300000A881C359D040A0FB35F8C056DF4FB88126
:10301000C05AD040B0FB36F8CC56DF4FE881C459D7
:10302000D040E0FB37F8832D837001F1813011F43B
:103030008BE201C08DE2C456DF4F68817981CC59A3
:10304000D040C656DF4FE881F981CA59D040099572
:10305000C257DF4F28813981CE58D0402F5F3F4F74
:10306000C257DF4F39832883CE58D040F11009C0B2
:10307000C257DF4FA880B980CE58D040A818B908F1
:1030800022C0C257DF4FE880F980CE58D0405401AB
:10309000AE18BF080150110917FD2DC0F501EE0D46
:1030A000FF1D8491C456DF4F68817981CC59D0408F
:1030B000C656DF4FE881F981CA59D0400995FFEF24
:1030C000EF1AFF0AE7CF7501E80CF91C015011094E
:1030D00017FD11C0C456DF4F68817981CC59D040AB
:1030E000D4018D914D01C656DF4FE881F981CA594F
:1030F000D0400995E8CFC057DF4FF881C059D04084
:10310000FF2309F4F1C821E0C21AD108D7FCECC8AA
:10311000C456DF4F68817981CC59D04080E2C656D1
:10312000DF4FE881F981CA59D0400995FFEFEF1AC6
:10313000FF0AE9CFC257DF4F88819981CE58D0402E
:10314000CC55DF4F0FB6F894DEBF0FBECDBFDF9179
:10315000CF911F910F91FF90EF90DF90CF90BF9094
:10316000AF909F908F907F906F905F904F903F9027
:103170002F9008959091C00095FFFCCF8A3041F0C8
:103180009091C00090649093C0008093C600089511
:103190009091C00090649093C0009DE09093C60011
:1031A0009091C00095FFFCCFEBCFCF939B01C091D6
:1031B000C1004091C10048604093C1004091C100EE
:1031C0004F794093C10040E050E06AEB78E10E9403
:1031D000F8108091C00086FFFCCFC093C100CF9152
:1031E0000895CF93C091C1009091C10098609093D1
:1031F000C1009091C1009F799093C10060E070E0A0
:103200000E94BA188091C00086FFFCCFC093C10015
:10321000CF910895CF93DF93CDB7DEB7FE013596FA
:1032200081919191BF010E94D518DF91CF910895AE
:103230001F93CF93DF931091C1002091C1002860AC
:103240002093C1002091C1002F792093C100FC017F
:103250008491EF012196882331F060E070E00E94B4
:10326000BA18FE01F5CF8091C00086FFFCCF109305
:10327000C100DF91CF911F910895AF92BF92CF927D
:10328000DF92EF92FF920F931F93CF93DF936C0126
:1032900085E0E82EF12C00E117E2C0E0D0E09AE0F2
:1032A000A92EB12CC601B8010E94FC1B6C0161154E
:1032B000710529F4209719F40130110529F480E3F0
:1032C000860F0E94F1182196C801B5010E94FC1BCF
:1032D0008B0181E0E81AF108E114F10419F7CE013D
:1032E000DF91CF911F910F91FF90EF90DF90CF90E2
:1032F000BF90AF900895CF93DF93EB010E94181910
:103300008AE30E94F118CE010E943D1983E795E0FF
:10331000DF91CF910C941819CF93DF93EC01CB017F
:10332000BA010E947B1986E795E00E941819CE0128
:103330000E9418198AE00E94F11881E090E0DF9164
:10334000CF9108950F931F93CF93DF93182F092FD9
:10335000EB01B901CA010E947B1985E695E00E9444
:103360001819CE010E9418190F931F938CE595E050
:103370009F938F930E940A190F900F900F900F90B8
:1033800081E090E0DF91CF911F910F910895505807
:10339000BB27AA270ED075C166D130F06BD120F0C3
:1033A00031F49F3F11F41EF45BC10EF4E095E7FB8E
:1033B00051C1E92F77D180F3BA17620773078407E9
:1033C000950718F071F49EF58FC10EF4E0950B2E61
:1033D000BA2FA02D0B01B90190010C01CA01A00167
:1033E0001124FF27591B99F0593F50F4503E68F1C2
:1033F0001A16F040A22F232F342F4427585FF3CF03
:10340000469537952795A795F0405395C9F77EF4D3
:103410001F16BA0B620B730B840BBAF09150A1F01C
:10342000FF0FBB1F661F771F881FC2F70EC0BA0FA2
:10343000621F731F841F48F4879577956795B7952A
:10344000F7959E3F08F0B3CF9395880F08F0992722
:10345000EE0F979587950895D9D008F481E00895E7
:103460000CD00FC107D140F0FED030F021F45F3F07
:1034700019F0F0C0511139C1F3C014D198F3992358
:10348000C9F35523B1F3951B550BBB27AA27621728
:103490007307840738F09F5F5F4F220F331F441F6D
:1034A000AA1FA9F333D00E2E3AF0E0E830D09150A5
:1034B0005040E695001CCAF729D0FE2F27D0660F92
:1034C000771F881FBB1F261737074807AB07B0E8D1
:1034D00009F0BB0B802DBF01FF2793585F4F2AF0E7
:1034E0009E3F510568F0B6C000C15F3FECF3983EC7
:1034F000DCF3869577956795B795F7959F5FC9F744
:10350000880F911D9695879597F90895E1E0660FCC
:10351000771F881FBB1F621773078407BA0720F045
:10352000621B730B840BBA0BEE1F88F7E0950895AE
:1035300004D06894B111D9C00895BCD088F09F57C9
:1035400090F0B92F9927B751A0F0D1F0660F771FEF
:10355000881F991F1AF0BA95C9F712C0B13081F0CF
:10356000C3D0B1E00895C0C0672F782F8827B85F17
:1035700039F0B93FCCF3869577956795B395D9F730
:103580003EF490958095709561957F4F8F4F9F4F3A
:103590000895E89409C097FB3EF490958095709546
:1035A00061957F4F8F4F9F4F9923A9F0F92F96E98F
:1035B000BB279395F695879577956795B795F11104
:1035C000F8CFFAF4BB0F11F460FF1BC06F5F7F4FA1
:1035D0008F4F9F4F16C0882311F096E911C07723B3
:1035E00021F09EE8872F762F05C0662371F096E8BC
:1035F000862F70E060E02AF09A95660F771F881F8B
:10360000DAF7880F9695879597F90895990F00082E
:10361000550FAA0BE0E8FEEF16161706E807F907A4
:10362000C0F012161306E407F50798F0621B730B3F
:10363000840B950B39F40A2661F0232B242B252BC0
:1036400021F408950A2609F4A140A6958FEF811D63
:10365000811D089597F99F6780E870E060E0089504
:103660009FEF80EC089500240A941616170618069A
:103670000906089500240A94121613061406050676
:103680000895092E0394000C11F4882352F0BB0F07
:1036900040F4BF2B11F460FF04C06F5F7F4F8F4F6A
:1036A0009F4F089557FD9058440F551F59F05F3FA5
:1036B00071F04795880F97FB991F61F09F3F79F054
:1036C00087950895121613061406551FF2CF4695D6
:1036D000F1DF08C0161617061806991FF1CF869558
:1036E0007105610508940895E894BB27662777273C
:1036F000CB0197F908958ADF08F48FEF08950BD076
:10370000C0CFB1DF28F0B6DF18F0952309F0A2CFC3
:10371000A7CF1124EACFC6DFA0F3959FD1F3950F71
:1037200050E0551F629FF001729FBB27F00DB11D45
:10373000639FAA27F00DB11DAA1F649F6627B00DD5
:10374000A11D661F829F2227B00DA11D621F739FBE
:10375000B00DA11D621F839FA00D611D221F749FCC
:103760003327A00D611D231F849F600D211D822F13
:10377000762F6A2F11249F5750408AF0E1F088235A
:103780004AF0EE0FFF1FBB1F661F771F881F915067
:103790005040A9F79E3F510570F05CCFA6CF5F3F28
:1037A000ECF3983EDCF3869577956795B795F7959A
:1037B000E7959F5FC1F7FE2B880F911D9695879522
:1037C00097F90895A29FB001B39FC001A39F700D08
:1037D000811D1124911DB29F700D811D1124911D19
:1037E00008950E94E21BA59F900DB49F900DA49F89
:1037F000800D911D1124089597FB072E16F4009457
:1038000007D077FD09D00E94321C07FC05D03EF49A
:10381000909581959F4F0895709561957F4F08957C
:10382000A1E21A2EAA1BBB1BFD010DC0AA1FBB1FC4
:10383000EE1FFF1FA217B307E407F50720F0A21B36
:10384000B30BE40BF50B661F771F881F991F1A94A3
:1038500069F760957095809590959B01AC01BD01CD
:10386000CF010895AA1BBB1B51E107C0AA1FBB1FB4
:10387000A617B70710F0A61BB70B881F991F5A95FC
:10388000A9F780959095BC01CD010895F894FFCFDC
:103890000000070620003C0188016801200020008C
:1038A00000300168016801000000000032000000E3
:1038B0005E010000FE3F3F3F003C4E554C4C3E0039
:1038C00018032F03370338033C033903E402EA02E9
:1038D000F7020C03ED023903303132333435363719
:1038E0003839414243444546303132333435363736
:0838F00038396162636465660A
:00000001FF
